:020000040800F2
:1000000000AA0120E5250008E1250008211E0008BE
:10001000E1250008E1250008E125000800000000B6
:10002000000000000000000000000000E1250008C2
:10003000E125000800000000E1250008E125000896
:10004000E1250008E1250008E1250008E125000878
:10005000E1250008E1250008E1250008E125000868
:10006000E1250008E1250008E1250008E125000858
:10007000E1250008E1250008E1250008E125000848
:10008000E1250008E1250008E1250008E125000838
:10009000E1250008E1250008E1250008E125000828
:1000A000E1250008E1250008E1250008E125000818
:1000B000E1250008E1250008E1250008E125000808
:1000C000E1250008E1250008E1250008E1250008F8
:1000D000E1250008E1250008E1250008E1250008E8
:1000E000E1250008E1250008E1250008E1250008D8
:1000F000E1250008E1250008E1250008E1250008C8
:10010000E1250008E1250008E1250008E1250008B7
:10011000E1250008E1250008E1250008E1250008A7
:10012000E1250008E1250008E1250008E125000897
:10013000E1250008E1250008E1250008E125000887
:10014000E1250008E1250008E1250008E125000877
:10015000E1250008E1250008E1250008E125000867
:10016000E1250008E1250008E1250008E125000857
:10017000E1250008E1250008E1250008E125000847
:10018000E1250008E1250008E1250008E125000837
:10019000E1250008E1250008E1250008E125000827
:1001A000E1250008E1250008E1250008E125000817
:1001B000E1250008E1250008E125000861070008A5
:1001C0006D070008E125000800000000E125000897
:1001D000E1250008E1250008E1250008E1250008E7
:1001E000E1250008E1250008E1250008E1250008D7
:0801F000E1250008E1250008EB
:0801F8009C0000000100000062
:1002000053B94AB9002908BF00281CBF4FF0FF317D
:100210004FF0FF3000F03CB882B0EC462DE90050C2
:1002200000F01EF8DDF804E002B00CBC704700BF1F
:100230002DE9F041904606460F461D46069C00F00B
:1002400029F808FB01FC8646A8FB002300FB05C536
:10025000B21A2B4467EB0303C4E90023BDE8F08125
:100260002DE9F8431D46174680468946089E00F052
:1002700053F900FB05F3A0FB074507FB0137B8EB7B
:1002800004043D4469EB0505C6E90045BDE8F88373
:10029000704700BF00292DE9F047C0F2A280002678
:1002A000002BC0F298808C4690469E461546044628
:1002B0000F46CBBB8A4256D9B2FA82F33BB1C3F1A7
:1002C00020029F409D409C4020FA02F21743280CD8
:1002D000220C1FFA85FEB7FBF0F100FB11770EFB35
:1002E00001F342EA0747BB4207D97F1980F0018139
:1002F000BB4240F2FE8002392F44FF1AA4B2B7FB82
:10030000F0F300FB13770EFB03FE44EA0747BE45FC
:1003100006D97F1980F0EB80BE4540F2E880023BB1
:1003200043EA0143002203E08B420FD90022134627
:10033000341C4FF0000518BF0124604265EB4501F5
:100340005840514000196941BDE8F087B3FA83F283
:10035000002A40F08380804540F2CD808B42C0F07F
:10036000CA801346E4E712B90123B3FBF2F5B5FAEC
:1003700085F2002A3BD1781B4FEA154E1FFA85FC07
:100380000122210CB0FBFEF80EFB18000CFB08F359
:1003900041EA0047BB4208D97F1980F0B080BB42D8
:1003A00040F2AD80A8F102082F44FF1AA4B2B7FBB7
:1003B000FEF30EFB13770CFB03FC44EA0747BC4536
:1003C00006D97F1980F09980BC4540F29680023BA7
:1003D00043EA0843ACE752426FEA060663EB430385
:1003E00061E740424FF0FF3661EB410158E795402D
:1003F000C2F1200107FA02F34FEA154ECF4024FA6A
:1004000001F194401FFA85FC1943B7FBFEF24FEA55
:1004100011480EFB12770CFB02F348EA0747BB4278
:1004200005D97F1971D2BB426FD9023A2F44FF1A06
:1004300089B2B7FBFEF80EFB18770CFB08F041EA17
:100440000743984206D95B1961D298425FD9A8F157
:1004500002082B44181A48EA024292E7C2F1200728
:1004600003FA02FE08FA02F5914028FA07F32CFA83
:1004700007FCF84043EA0E0E08434FEA1E48070CFB
:100480001FFA8EFABCFBF8F908FB19CC0AFB09F13C
:1004900047EA0C4C614507D91CEB0E0C32D2614582
:1004A00030D9A9F10209F444C1EB0C0C80B2BCFBB9
:1004B000F8F308FB13CC0AFB03FA40EA0C418A4527
:1004C00006D911EB0E0125D28A4523D9023B71448E
:1004D00043EA0943CAEB0101A3FB0589494503D35C
:1004E00003D19440444500D2013B002220E7013B68
:1004F00016E7013901E701231AE7013B68E708F134
:10050000FF3852E709F1FF39CEE7013A8FE708F1EA
:10051000FF389FE7013BDBE72DE9F043002B40D19B
:100520008A42044615464AD9B2FA82F30F464BB1C5
:10053000C3F12006994000FA03F402FA03F5F040F3
:1005400040EA0107290C260C1FFA85FEB7FBF1F0E3
:1005500001FB10770EFB00F246EA07439A4207D9E7
:100560005B1980F0EA809A4240F2E78002382B441F
:100570009A1AA4B2B2FBF1F301FB13220EFB03FEA5
:1005800044EA0242964506D9521980F0DA8096452F
:1005900040F2D780023B43EA004000263146BDE8E6
:1005A000F0838B4244D8B3FA83F6002E45D18242C1
:1005B00040F2BF808B42C0F0BC803046EEE712B9FB
:1005C0000125B5FBF2F5B5FA85F2002A7BD14A1B6D
:1005D0002F0C1FFA85FE0126230CB2FBF7F007FB58
:1005E00010220EFB00FC43EA02418C4507D9491951
:1005F00080F0A1808C4540F29E8002382944CCEBEB
:100600000101A4B2B1FBF7F307FB13110EFB03FECC
:1006100044EA0144A64506D9641980F09080A645B5
:1006200040F28D80023B43EA00403146BDE8F08352
:10063000002630463146BDE8F083C6F12005B340C0
:1006400002FA06F701FA06F4EA40E94020FA05F555
:100650001A4325434FEA124C4FEA154E93B2B1FBB1
:10066000FCF80CFB181103FB08F44EEA01418C4224
:1006700006D9891869D28C4267D9A8F102081144B9
:10068000091BADB2B1FBFCF40CFB141103FB04FE1F
:1006900045EA01439E4505D99B1854D29E4552D93F
:1006A000023C134444EA0844CEEB0303A4FB07894D
:1006B0004B4503D351D1B04040454ED20026601E79
:1006C0003146BDE8F083C2F12006954001FA02F3FD
:1006D00000FA02F42F0CF140F0401FFA85FEB1FB46
:1006E000F7F6184307FB16110EFB06F24FEA104C03
:1006F0004CEA01439A4205D95B1929D29A4227D97B
:10070000023E2B449B1A80B2B3FBF7FC07FB1C3361
:100710000EFB0CF140EA0343994206D95B1919D24A
:10072000994217D9ACF1020C2B445A1A4CEA0646EE
:1007300052E7012032E7013861E7013818E7013B51
:1007400071E7013B27E7013CACE708F1FF3897E789
:10075000013ED7E70CF1FF3CE7E7204600261DE706
:10076000014800F0E2BF00BFE82B0008014801F09B
:1007700044B800BFE82B0008014800F005BE00BFE8
:10078000E82B000837B50024012002F009FA019097
:100790002546E0B200F046F801AA08B910551DE060
:1007A000135D042B0BDD174800F03CF9019800F0B5
:1007B00040F90120002102F0E3F9002020E001339C
:1007C000DBB2042B135509D90F48012500F012F9AB
:1007D000204600F02EF90D4800F024F90134042CD5
:1007E000D7D1019C3CB10A4800F004F9204600F042
:1007F00020F900F08FF80120214602F0C1F92846C7
:1008000003B030BDD1650008FD650008086600082A
:100810001266000808B500F083FB80F00100C0B24A
:1008200008BD000008B50C22044B02FB003000F0AC
:1008300099FC80F00100C0B208BD00BF882C000800
:1008400010B5002401F096F8054820440C34017AD4
:1008500000F06EFC302CF7D1BDE8104001F08BB8F1
:10086000882C0008044BDA691106FBD59862DA6916
:100870001206FCD5704700BF0048004070B5214DFE
:100880008AB02148082101F077F828464FF48021EA
:100890001E4C01F071F82B68642623F0010394E8E4
:1008A00007002B600C348DE8070000216846022207
:1008B0000B4600F01FFC03AB94E8070083E8070039
:1008C00000211846022200240B4600F013FC06A863
:1008D00002F07CF8089821460D4A70430023FFF788
:1008E0008FFCC0F3420320F00F000004000C1843FB
:1008F0000D23B0FBF6F0E8606C60AC602B600AB0D2
:1009000070BD00BF00480040000C0240B82C000839
:1009100040420F002DE9F043334D83B02C6800AF07
:1009200004F12E0304F1270823F00703ADEB030DB8
:1009300050238DF8003021236E460DF106028DF80C
:10094000013000238DF8023003238DF8033004F1C9
:1009500021035BBAADF80430244B03F11C0153F8BA
:10096000040B8B4242F8040BF9D11B7804F12309E4
:1009700006F123001E491370224602F021F9314688
:100980004A46002001F072FD07F1080304F5927455
:10099000314643F8040D42461868FE23B4FBF3F3D6
:1009A000434446F80900073323F00703ADEB030D7A
:1009B00068466E4601F032FD044655206C44FFF750
:1009C00051FFA64207D016F8010B552808BF00209A
:1009D000FFF748FFF5E75520FFF744FF00230C37EA
:1009E0002B60BD46BDE8F08338000020D02C000805
:1009F0003C00002010B5441E14F8012F7AB10849BC
:100A00000B68FF2B0BD80A2A02D1FFF783FFF3E70D
:100A10000D2A1FBF581C5B1808601A71ECE710BD47
:100A20003800002008B5FFF7E5FFBDE80840FFF7F4
:100A300071BF1FB50C2201A901F046FD01A8FFF707
:100A4000D9FF05B05DF804FB07B502A9012201F842
:100A5000010D042000F096F903B05DF804FB0021BD
:100A600002200A4600F08EB910B540F2F51400F0ED
:100A7000B9F850B1013C04D10548FFF7D3FF204637
:100A800010BD642001F012FDF1E7012010BD00BF90
:100A90003E66000810B5074C43F2CD71064848F693
:100AA000B803224601F058FD01462046BDE810403B
:100AB00000F0E4B83C010020ED2C000810B500F077
:100AC00099F8FFF7E7FF08B9154816E0002400F091
:100AD00039F9FFF7C4FF0120FFF7B6FFFFF7C4FFA6
:100AE00078B1002103200A4600F04CF90D48FFF7C9
:100AF00081FF2046FFF79DFF0B48BDE81040FFF740
:100B000091BFFFF7C7FF0028DED001340B2CE2D1E4
:100B10000648FFF787FFBDE81040FFF7A0BF00BF02
:100B2000616600087C66000897660008A1660008F8
:100B300008B5FFF799FF0120FFF786FFFFF794FF45
:100B4000002103200A46BDE8084000F01BB9000060
:100B50002F2307B54A1C58430B4B00EB52001A7861
:100B6000B0FBF1F0C0B282420AD002A91870042290
:100B700041F8040D012000F005F90220FFF764FFA1
:100B800003B05DF804FB00BF0000002007B502A918
:100B9000042241F8040D012000F0F4F80320FFF7CF
:100BA00053FF03B05DF804FBFFF759BF0C4B014442
:100BB00030B51C68884207D022689568AD07FCD51F
:100BC00010F8015B1573F5E71B681A68936813F456
:100BD000C05FFBD10A20BDE8304001F067BC00BF18
:100BE000382C0008024B1868403000F0BBBA00BF38
:100BF000382C000838B5204B012200211C6804F174
:100C00002005284600F048FA0021284600F05EFA48
:100C100004F1380000F0A0FA04F1400000F09CFA62
:100C2000012104F12C000A4600F036FA002104F1FB
:100C3000080001220B4600F05DFA0021012204F1B8
:100C400014000B4600F056FA6068012101F070FFB5
:100C50006068002101F06CFF94E8030000F08CFE56
:100C600023684CF207321A604FF4B8525A601A687F
:100C700042F040021A6038BD382C00082B4B2DE999
:100C8000F7431C68814601208846E36A04F1200787
:100C900004F12C060093236B019301F00BFC384602
:100CA000012100F013FA0021304600F00FFA012074
:100CB00001F000FC684600F055FA054620B11C48DA
:100CC0000025FFF7AFFE2CE030460121383400F05C
:100CD000FDF9012001F0EEFB204600F043FA064644
:100CE00008B114481BE0684600F03CFA054608B914
:100CF000114814E0012001F0DDFB48464146FFF7B2
:100D000055FF3846314600F0E1F90C480921FFF75C
:100D10004DFF204600F026FA054610B90848FFF7B7
:100D200081FE284603B0BDE8F08300BF382C0008E0
:100D3000C0660008DC660008F6660008BA640008B1
:100D40001267000808B5022001F0B4FB0A4B1B68CB
:100D500093F8483043B10948FFF764FE012000F0E2
:100D6000D9FD022001F0A6FB0548FFF75BFE01203C
:100D7000BDE8084000F0C8BD382C00083367000803
:100D80004F6700080F4BF7B51C6802AD0F460121F5
:100D9000203405F8010D1646204600F097F964202E
:100DA00001F084FB28460121FFF700FF1EB1384601
:100DB0003146FFF7FBFE2046002100F087F903B023
:100DC000F0BD00BF382C0008F0B50746ADF2044D69
:100DD0000E460C460025B919B4F5806F6846A1EBA4
:100DE00004010DD94FF48062A4F5806400F0D8F8B6
:100DF000284669464FF4806201F038FB0546EAE771
:100E0000224600F0CDF869462246284601F02EFB26
:100E10000DF2044DF0BD08B5202001F0A1FD002821
:100E2000FAD108BD08B5022001F09AFD0028FAD0D9
:100E30000220BDE8084001F09DBD00B58DB06846B8
:100E400001F017FD0023684600934FF480730A9366
:100E500035230B9301F03EFDFFF7E4FFFFF7DBFFC7
:100E60000DB05DF804FB000030B5002495B02A48B1
:100E7000022100F081FD294D0021032228190C34A4
:100E80000B4600F037F9482CF5D1002105F1480058
:100E900000240A4600F000F9002105F148004FF453
:100EA000407500F013F901A801F0DAFC102301A845
:100EB00002940193172303940593049406940794D2
:100EC00001F0E6FC012001F029FDFFF7B6FF08A8BC
:100ED00001F0CFFC662308A808941393129501F043
:100EE000F9FCFFF79FFF08A801F0C3FC992308A8AD
:100EF00008941393129501F0EDFCFFF793FF4CF269
:100F0000503001F0D3FAFFF798FF0348022100F0B8
:100F10003DFD15B030BD00BF001000A0C464000846
:100F200030B502218DB01C4800F026FD022001F0F2
:100F300009FD684601F09DFC4FF080636846009310
:100F40004FF0407304934FF440730A93AF230B9315
:100F500001F0C0FCFFF766FF01F0FCFC054601F064
:100F6000F9FC044601F0F6FC240244EA004040EAA1
:100F70000504FFF750FF094B9C4204D02046002493
:100F8000FFF757FD00E001240348022100F0FEFCBA
:100F900020460DB030BD00BF001000A020BB1800DF
:100FA00070B515468CB004460E461B48022100F071
:100FB000E3FC681E01F0C6FC684601F05AFC4FF0E5
:100FC00080636846254400934FF0407304930A23DE
:100FD00005934FF4406309934FF440730A934FF421
:100FE000005308930B230B9301F074FC304601F07F
:100FF000A1FCAC4204D001F0ADFC04F8010BF8E711
:10100000022001F0B7FCFFF706FF0348022100F0C1
:10101000BDFC0CB070BD00BF001000A0034A136BF4
:1010200023F4FF6323F00703136370470038024083
:1010300000F13F4000F57E00C0F387200A280AD85F
:10104000054A135C591C11542BB9044901230A6B3E
:10105000834013430B637047F4890020003802403B
:1010600000F13F4000F57E00C0F387200A280DD82C
:10107000074A135C53B1013BDBB2135433B9054942
:1010800001230A6B834022EA03030B63704700BF0E
:10109000F489002000380240436813B5009301230F
:1010A000044600688DF8043000238DF805208DF883
:1010B00007308DF80610FFF7BBFF2068694601F086
:1010C00059FB2068FFF7CCFF02B010BD38B5037A9A
:1010D00004460D460BB981F001052068FFF7A8FF13
:1010E0002068A1882A4601F083FB2068BDE83840CB
:1010F000FFF7B6BF13B5044640688DF8073000907F
:1011000002208DF805208DF8040020688DF8061067
:10111000FFF78EFFA27A2068218901F06DFB20681D
:10112000694601F027FB2068FFF79AFF02B010BD67
:10113000002313B5044601934368006800938DF8BB
:101140000710FFF775FF2068694601F013FB206860
:10115000FFF786FF02B010BD036813B10021FFF74F
:10116000E7BF704738B504460068FFF761FFA18804
:10117000206801F037FB05462068FFF771FF281C47
:1011800018BF012038BD1FB5836804460093C368AB
:1011900068460193FFF7E0FF636902A80293A36921
:1011A0000393FFF7D9FF04B010BD10B50446012129
:1011B000083002220023FFF79DFF04F114000121F3
:1011C00002220023BDE81040FFF794BF0368DB69EB
:1011D00010B5044673B9C36A63B10A2001F06AF915
:1011E0002046FFF7D0FF2046E36A012198471420EC
:1011F00001F060F92046FFF7D8FF2046BDE8104017
:1012000000F0E0B910B5044600F04FFA48B10A20EA
:1012100001F050F9204600F048FA80F00100C0B219
:1012200010BD012010BD30B5044687B0C36A00214F
:101230009847A3680021012500936846E3680A46A1
:101240008DF808500193FFF727FF68460021FFF74C
:101250003DFF6369002103A80393A3690A468DF843
:1012600014500493FFF718FF03A80021FFF72EFF87
:1012700007B030BD10B5044600F00AFA2368DB69F8
:1012800033B9E36A4BB12046BDE81040FFF7CBBF4E
:101290002046BDE81040FFF776BF10BD10B50446EC
:1012A000FFF7E8FF2046BDE81040FFF78FBF0000C2
:1012B0002DE9F3419846036804460E46DB6917465C
:1012C0000BB900205BE000F0F0F9B8B925681422F2
:1012D0000021284601F07FFC9DF828306F802046D1
:1012E0006B71089B2E71AB60099B85F806802B61A2
:1012F00000F0ECF9236800229A6111E02046FFF724
:10130000CDFF2046FFF77EFF0028DFD1D9E79A699D
:10131000B2F57A7F23DA013202209A6101F0CAF82D
:10132000204600F0DFF90122236883F82020154AC7
:101330000192019A511E01911AB193F82020002ABE
:10134000F7D1002283F82020019A42B11D7D05F0DB
:10135000FD02012ADBD16B1E5D425D4103E00025E9
:10136000204600F0A8F923680022204683F82020B8
:10137000FFF748FF10B92046FFF790FF284602B05C
:10138000BDE8F08180841E0010B5044618B90E48EF
:10139000A92101F00BF800212422006801F01BFCB8
:1013A000204600F0CBF8236A2BB1002104F1200085
:1013B0000A46FFF771FEE36A23B12046BDE81040FC
:1013C000FFF731BF10BD00BFA567000810B5044688
:1013D00018B90848B62100F0E9FF00680368DB6926
:1013E0000BB9FFF7F3FE23681A68D3690133D361A1
:1013F00010BD00BFA567000808B518B90748BF2190
:1014000000F0D4FF00680268D36933B1013BD361B7
:101410001BB9BDE80840FFF72DBF08BDA567000850
:101420001FB50C46114618B90A4840F28D1103E069
:1014300023B908484FF4C77100F0B8FF82888DE8DF
:101440000A000021234602910068FFF731FF04B033
:1014500010BD00BFA567000813460122FFF7E0BFDB
:101460001FB50C46114618B90A484FF4D77103E06E
:1014700023B9084840F2AF1100F098FF82888DE848
:101480000A0000230121029323460068FFF710FFA2
:1014900004B010BDA567000807B502AB03F8012D25
:1014A0000122FFF7DDFF03B05DF804FB03680022B3
:1014B000197583F82020704710B504686388227975
:1014C000C3F3090322B92278012A18BF43F48063C9
:1014D000A268E468121BFF2A95BF120443F0FF7351
:1014E00002F47F0243F4803398BF134309B143F4FD
:1014F000005342681268536010BD43681B681A6845
:1015000022F0D60210B51A605A6842F480425A603E
:1015100008220368BDE810401A70FFF7C7BF0368D0
:10152000012110B50446586801F0F6FA002123683D
:10153000BDE81040586801F0EFBA000043685A7BDC
:1015400053B2002B30B506DA02F00F021B4B1344E6
:10155000C0221A7606E003F16043C02203F561431E
:1015600083F8002343689A7B53B2002B06DA02F01B
:101570000F02124B1344C0221A7606E003F16043B7
:10158000C02203F5614383F8002350F8045F0C4C3C
:101590006B7B59B203F01F020123490903FA02F2DF
:1015A00044F82120AA7B51B202F01F02490993405E
:1015B00044F82130BDE83040FFF7B1BFFCEC00E05B
:1015C00000E100E043682C499A688A42F0B507467A
:1015D00087B004D929485121294A00F0DBFE294966
:1015E0008A4205D91C7B34B1012C07D000F0E8FEFB
:1015F0000124254603E00924102500E0022502A865
:1016000001F0E4F979686019049A8B684343B2FBEE
:10161000F3F603FB162303B9013E0F2E03D9174837
:10162000702100F0C3FE03C900F0A6F97B684FF0FB
:10163000000100221B68013D66F307110192013C85
:101640008DF804508DF8071019688DF8054021F0C9
:10165000010119600C49186801401960019919616C
:101660009A60DA601A6842F001021A60074A596803
:101670000A405A6007B0F0BD801A0600BE67000835
:10168000DB670008A0860100001F30FF008000F823
:1016900010B5044654F8043F93E8030000F076F9CF
:1016A0002046BDE81040FFF73ABF43681B689869C1
:1016B000C0F3C030704743681B681A6822F0D60236
:1016C0001A605A6842F480425A60704703685A7937
:1016D0000AB9012204E01A790AB9052200E00622BB
:1016E0001A70704743681B681A6842F0D20210B53E
:1016F0001A60026814791CB9196841F00401196074
:10170000117801290CD15288012CC2F309020CBFB7
:101710004FF08071002142F490320A435A6010BDAC
:101720000121BDE81040FFF7C7BE38B54368054644
:101730001C6803681A78013A072A5BD8DFE802F0D0
:10174000045A5A5A223B5A57A269910701D59A79ED
:10175000A2621A793AB9A26952060FD50522284623
:1017600001211A7008E0012A08D1A269100605D5E6
:101770000622284600211A70FFF79EFEA369D906AB
:101780003AD525E0A269520705D5DA681969501CD7
:10179000D860636A8B54A3691B0603D528460021D1
:1017A000FFF78AFEA369580626D528460121BDE821
:1017B0003840FFF7A2BEA269910705D5DA6819691A
:1017C000501CD8608B5CA362A16911F0100109D094
:1017D000E3692846022143F01003E361BDE8384085
:1017E000FFF764BEA3691A06DCD52846D8E7A369CB
:1017F000DB0701D400F0E4FD38BD43681B689A693B
:10180000D20503D5DA6942F48072DA619A6951052A
:1018100003D5DA6942F48062DA619A69920503D5E8
:10182000DA6942F40072DA610321FFF766BE000054
:10183000094B70B51C680D4606462046FFF7C6FDED
:101840002A4631462046FFF707FE05462046FFF7A9
:10185000D3FD284670BD00BF1C2C0008094B70B595
:101860001C680D4606462046FFF7B0FD2A46314665
:101870002046FFF711FE05462046FFF7BDFD28462E
:1018800070BD00BF1C2C000837B500F073F81B4872
:1018900001210222FFF700FC194801210222FFF773
:1018A000FBFB00F068F800200DF10701FFF7C0FF17
:1018B0009DF80750012D1DD114200DF10701FFF7F0
:1018C000B7FFA8B10F4C237813B1013323700FE099
:1018D0009DF80710142021F0060141F002018DF857
:1018E0000710FFF7BBFF18B10320257000F0E2FDE1
:1018F000012000E0002003B030BD00BF18650008E3
:1019000030650008FF89002001460148FFF7DEBB73
:101910001865000870470000B0F1804F08B503D289
:101920000D48302100F042FD0C4B98420ED903F5D2
:10193000803398420CD9B0F1A04F0BD3084A094B21
:10194000B0F1204F34BF1846104608BD064808BD08
:10195000064808BD064808BDFC670008FFFF0040B8
:10196000892A0008712A0008A12A0008B92A00085B
:10197000592A00087047704710B50C46FFF7CCFF96
:10198000012103462046BDE81040184710B50C461B
:10199000FFF7C2FF002103462046BDE8104018476C
:1019A00038B5104C05464FF080512046FFF7E4FF54
:1019B00045B154E8003F43F4807344E80032002A04
:1019C00008D0F6E754E8003F23F4807344E800327F
:1019D000002AF7D103484FF08051BDE83840FFF7A7
:1019E000D5BF00BF00700040024B5868C0F34000F4
:1019F000704700BF00700040024A136843F00803BC
:101A00001360704700700040B0F1006F10B50446DD
:101A10000BD20C48FEF7EEFF2046FFF70AF80A4803
:101A2000FFF700F84FF0FF3010BD084B002053F8CF
:101A3000042BA24202D81A68944202D301300B2828
:101A4000F5D110BD1B680008246800083C6500083B
:101A50002DE9F8430446174699460E46C1B3FFF7F1
:101A6000D3FF0546601E3044FFF7CEFF002D8046B1
:101A700031DB00282FDB461B01361FB10020314629
:101A80004A46B8472C4600F0D3FD44451EDCF320FF
:101A900000F0E4FD114B002133F8140000F016FEB5
:101AA00009280AD00E48FEF7A5FF2046FEF7C1FF21
:101AB000FEF730FF00F0CAFD0DE02FB1C5F10100C7
:101AC00031464A462044B8470134DEE700F0BEFD07
:101AD0000120BDE8F8830020BDE8F8836C650008AC
:101AE0003D6800082DE9F0410F461646804600F09B
:101AF0009FFD3E443C46F32000F0B0FDB44216D0BA
:101B0000C7EB0805254414F8011B284600F014FE15
:101B10000928F3D00848FEF76DFF2846FEF789FF35
:101B2000FEF7F8FE00F092FD0020BDE8F08100F025
:101B30008DFD0120BDE8F0815568000808B545F22B
:101B4000555000F06BFE042000F06EFE40F6FF7072
:101B500000F070FE002000F061FE4FF48050012183
:101B6000BDE8084000F058BD08B500F071FEBDE8C2
:101B7000084000F065BE08B57D2000F0E5FF0030AC
:101B800018BF012008BD4900FEF7E2BF2DE9F04370
:101B9000012185B005460020FEF7DAFF042000F0A1
:101BA00051FB01A8294600F0A7FB01A800F0B3FBF8
:101BB00008B93B4814E00C353A48FEF733FF029968
:101BC0002846FFF701F904463748FEF713FF204681
:101BD000FEF72FFFFEF79EFE039B9C4204D0334886
:101BE000FEF720FF012057E0029CDFF8E08030483C
:101BF000FEF718FF21462F4A002340460024FFF736
:101C000027FF029F2C484FEA5709FEF70BFFBC4203
:101C10001CD23E1B29486119B6F5803F28BF4FF4FE
:101C200080363246FFF7BCF908EB04002349324600
:101C3000FFF758FF18B92248FEF7F4FE06E009EB5B
:101C400054003946FEF784FF3444E0E71D48FEF7B0
:101C5000D1FE0298FEF7EDFE1B48FEF7CBFE1B49B6
:101C6000029A002000F002FC04461948FEF7C2FE6A
:101C70000398FEF7DEFE1748FEF7BCFE2046FEF78F
:101C8000D8FEFEF747FE039B9C4204D01248FEF7A5
:101C9000C9FE022000E0002005B0BDE8F08300BFCF
:101CA0006668000884680008A1680008B768000832
:101CB000DA680008871B0008F1680008008A002025
:101CC00008690008136900082169000800800008FD
:101CD0002A6900083D6900084369000810B5022020
:101CE00000F0C8FAD8B3042000F0C4FA044670B17A
:101CF0001B48FEF797FE042000F0B0FA022000F027
:101D0000ADFA4FF40040BDE8104000F0A7BA154806
:101D1000FEF788FE082000F0A1FA102000F09EFADD
:101D2000202000F09BFA402000F098FA2046FFF7B0
:101D30002DFF022807D1082000F084FA102000F0BF
:101D400081FA00F061FB042000F088FA022000F024
:101D500085FA4FF40040BDE8104000F073BA10BDA2
:101D60008E690008C469000810B52548FEF75AFEC0
:101D70004FF48000FFF70AFF10B102283AD809E0BB
:101D8000202000F06BFA402000F068FA802000F07C
:101D900059FA2FE0082000F055FA102000F052FA0E
:101DA000202000F067FA20B91648FEF73BFE2020FD
:101DB00007E0402000F05EFA58B91348FEF732FE03
:101DC000402000F03FFA4FF4007000F03BFA00F0C2
:101DD0001BFB0E480024FEF725FE082000F03EFA0B
:101DE000102000F03BFA202000F038FA402000F0EC
:101DF00035FA00E00124042000F030FA204610BD3E
:101E0000DF690008F9690008326A00086B6A000897
:101E100008B50248FEF706FE00F0FDFAA56A0008C4
:101E20001EF0040F0CBFEFF30880EFF30980FFF7FB
:101E3000EFBF704708B50120FEF7F4FC08B9002099
:101E40000FE00020FEF7EEFC0028F8D00220FEF79D
:101E5000E9FC0028F3D00320FEF7E4FC80F0010049
:101E6000C0B200F0010008BD1FB504460E48FEF7E1
:101E7000D9FD01A90C22204600F026FB01A8FEF79F
:101E8000D1FD2046FEF782FE0220FEF7CBFC044681
:101E90000220FEF7C7FCA04201D000F0B5FA0A20EC
:101EA00000F008FBF4E700BF9B6A00087FB5BF485D
:101EB0004FF08051FFF760FDFFF796FD044630B10B
:101EC000FFF79AFDBA48FEF7ADFD00F0A4FA4FF017
:101ED0008051B648FFF75AFDFEF74EFCFEF7CEFCE8
:101EE000B448FEF79FFDB448FEF79CFDB348FEF7EB
:101EF00099FDB348FEF796FDB248FEF793FDB24850
:101F0000FEF790FDB148FEF78DFDFFF7BDFC00F038
:101F1000BBF900F0DBF921460C2201A800F05BFEC2
:101F200000F0D0F901A90C2200F0CEFA01A8FEF7CA
:101F300079FDA748FEF776FDA548FEF773FD4FF43F
:101F4000804000F097F990B1A248FEF76BFD4FF486
:101F5000804000F083F9082000F080F9102000F0A4
:101F60007DF9202000F07AF9402000F077F9FEF7A3
:101F70007BFFFEF765FCFFF787FCFEF79FFDFEF792
:101F8000D7FDFEF7FFFB08B1934803E0FEF742FCE4
:101F900010B19248FFF768FF00F084F9802000F04C
:101FA00069F918B1802000F059F94BE04FF4003086
:101FB00000F060F920B14FF4003000F04FF943E039
:101FC000FFF738FF68B141F288348548FEF72AFDF3
:101FD000FFF730FF78B1012000F06CFA013CF7D137
:101FE00032E0804B0CCB013301D0013203D17E486B
:101FF000FEF718FD28E0FFF7BEFD48B3FFF7BBFD75
:1020000010B17A48FEF70EFD4FF4007000F032F97F
:1020100010B17748FEF706FD4FF4007000F01EF98E
:10202000102000F027F9002800F0F8807148FEF732
:10203000F9FC082000F012F9102000F00FF9FFF76A
:1020400093FE98B96C48A5E76C48FEF7EBFCF6E701
:102050004FF4007000F00EF90028CFD1082000F0F6
:10206000FDF8102000F0FAF8FFF738FE4FF40050AA
:1020700000F000F904464FF4805000F0FBF84000F7
:1020800040EA8400C4B24FF4006000F0F3F820434B
:10209000C0B20728C3B20DD14FF4006000F0DEF8E3
:1020A0004FF4805000F0DAF84FF4005000F0D6F80A
:1020B00053486FE701334FF40060DBB2023B052B5E
:1020C00011D8DFE803F00C1003100C1000F0C6F874
:1020D0004FF4805000F0C2F84FF4005003E000F0DD
:1020E000BDF84FF4805000F0ADF84648FEF79AFC7A
:1020F000FFF724FDFFF738FDFEF790FF394B42480C
:102100005D681E68FEF776FC2846FEF792FC3F48A5
:10211000FEF770FC0022930001324FF0FF3103F113
:102120006043082A03F56143C3F88010C3F88011A7
:10213000F1D1374B4FF4801200241A634FF48062C0
:102140005C639C631A645C6400F01AFC31480121F2
:1021500000F0BEFC21462F4800F0BAFCF32001211C
:1021600000F0C2FC2146F32000F0BEFC0320012158
:1021700000F0C6FC2146032000F0C2FC6FF4A05022
:10218000012100F0C9FC21466FF4A05000F0C4FC0E
:102190002148012100F0CCFC1F48214600F0C8FC7A
:1021A00063B64FF0FF3EB546284700BF00700040C1
:1021B000B06A0008BD6A0008C46A0008516B0008D4
:1021C000E86B0008696C0008EA6C00086D6D000897
:1021D000C36A0008EA6D0008014550FE024550FE42
:1021E000176E000800800008526E0008656E000837
:1021F0007D6E00089D6E0008034550FE116F0008BB
:10220000044550FE306F0008426F0008566F00080A
:10221000003802400010E022B379F764082000F093
:1022200029F820B10548FEF7FDFB102003E0044823
:10223000FEF7F8FB082000F005F815E7C56E00086A
:10224000EB6E000810B50446002000F0A9FC40EA3F
:1022500004010020BDE8104000F092BC10B5044617
:10226000002000F09DFC20EA04010020BDE81040A1
:1022700000F086BC10B50446002000F091FC20421E
:1022800014BF0120002010BD08B50120FFF788FB16
:102290000120FFF7EFFF20B90121BDE8084000F061
:1022A0006FBC08BD08B50648FEF7A4FB002000F08F
:1022B00077FCFEF7BEFBBDE80840FEF72BBB00BF76
:1022C0005E6F0008022000F06BBC000008B5FFF74D
:1022D000F9FF0449884204D00220BDE8084000F01C
:1022E0004FBC08BD8BB8185808B50248FEF79AFBDA
:1022F00000F08AF86A6F00081FB504460C2201A896
:10230000FEF74EFE01AB03CB206018686160A06051
:10231000204604B010BD0068A0F10C03584258419B
:102320007047000080B51746064610480D461C460B
:10233000FEF760FB3846FEF75DFB0D48FEF75AFBE3
:102340003046FEF757FB0B48FEF754FB2846FEF7D6
:1023500070FB2CB10848FEF74DFB2046FEF74AFB08
:102360000648FEF75FFBFFF7BFFF00BF876F00085F
:102370006A6D0008906F00086B6D0008C36A000862
:102380001FB506AA52F8044B039200921A46234640
:10239000FFF7C8FF0CB41FB506AA52F8043B03921E
:1023A0000092014AFFF7BEFF926F0008002307B5B5
:1023B00072460093014BFFF7E3FF00BF996F0008DF
:1023C0007446064808B5FEF715FB2046FEF731FBBC
:1023D0000348FEF727FBFFF787FF00BFA16F000848
:1023E000C36A0008BFF34F8F0549064BCA6802F461
:1023F000E0621343CB60BFF34F8F00BFFDE700BF28
:1024000000ED00E00400FA0508B5FEF7CDFB00F092
:10241000AFFBFFF7E7FF08B5FFF7E4FFF0B50646AF
:10242000002401202546034694421DD011F804C023
:1024300000F1010EBCF1000F03D17355774605463C
:102440000DE00133774606F800C0DBB2FF2B07D161
:1024500002F1FF3C644506D07355871C7546012385
:1024600001343846E0E770467355F0BD30B5C9B168
:10247000C0430A44914213D011F8013B0A4D83EA4C
:10248000000404F00F0455F8244084EA101080EA98
:10249000131303F00F0355F8233083EA1010E9E714
:1024A000C04330BD084630BD8465000800010138D6
:1024B000FDD1704710B504462CB14FF47A70013C41
:1024C000FFF7F4FFF8E710BD0A2A10B504DC114845
:1024D000BDE81040FEF7A6BA30230C461C2204F8D3
:1024E000023B78234B700F2393400340D340092BCA
:1024F00001D8303302E00F2B02D85733DBB200E0B3
:102500002023043A04F8013B131DECD100238B7205
:1025100010BD00BFDB6F000808B5826843689342B6
:1025200003D304481421FFF741FF0268591C41609E
:10253000D05C08BDF16F000843688268934210B513
:1025400003D304481921FFF731FF02685C1C446083
:10255000D15410BDF16F0008F0B587B00E460746A4
:10256000154600210C2268461C4600F034FB002171
:102570000C2203A80296009700F02DFB68460395F5
:102580000594FFF7C9FF06466846FFF7C5FFB0424E
:10259000014601D003A808E06846FFF7BDFF0446E6
:1025A000D8B1012804D103A83146FFF7C5FFEBE7F6
:1025B000030608D504F07F046846FFF7ADFF40EA44
:1025C000042000F18004A4B20025A542DCDA03A8AF
:1025D0000021FFF7B1FF0135F7E7049807B0F0BD20
:1025E000FEE700000748084A0849121A08B500F03B
:1025F000E7FA0748074A0021121A00F0ECFAFFF741
:1026000055FC00BF000000201400002004700008EA
:1026100014000020008A0120044B9A6809B110437D
:1026200001E022EA00009860704700BF002004E04B
:10263000044B1A69002A04DA034A5A6002F188320C
:102640005A607047003C024023016745024A136903
:1026500043F0004313617047003C0240014BD860D7
:10266000704700BF003C02400E4BDA68D20310D422
:10267000DA68D1060FD4DA68D2050ED4DA6812F01F
:10268000E00F0CD1DB6813F0020F14BF0820092003
:1026900070470120704706207047022070470720CE
:1026A000704700BF003C0240092307B58DF8073092
:1026B000FFF7DAFF8DF807009DF80730012BF7D000
:1026C0009DF8070003B05DF804FB000070B50646F6
:1026D00041B1012908D002290CBF4FF400754FF415
:1026E000407503E00D4601E04FF48075FFF7DCFF15
:1026F00009281ED10F4C236923F4407323612169FB
:1027000029432161236923F0F8032361236943F0FE
:1027100002031E432661236943F480332361FFF7DC
:10272000C3FF236923F002032361236923F0F80325
:10273000236170BD003C024070B505460E46FFF7B0
:10274000B3FF092813D10A4C236923F44073236192
:1027500023692361236943F0010323612E70BFF3D2
:102760004F8FFFF7A1FF236923F00103236170BDA1
:10277000003C0240F0B500220E680123934003EABA
:10278000060E9E452AD1550003230468AB40DB4367
:102790001C4004600C79076804FA05FC013C4CEA13
:1027A0000707012C076011D884684F791C40AF409F
:1027B0008460846827438760446824EA0E04446088
:1027C0008C7947689440A4B23C434460C468234079
:1027D000C360CB79C468AB402343C3600132102A85
:1027E000CBD1F0BD0369194214BF0120002070470E
:1027F00002B909048161704701F00703C9089B0011
:1028000000EB81000F219A40994010B5046A24EA38
:1028100001010162016A1143016210BD014B1860A0
:10282000704700BF00300040014B5860704700BF48
:1028300000300040014B9860704700BF00300040FE
:102840004AF6AA22014B1A60704700BF00300040D0
:102850004CF6CC42014B1A60704700BF003000407C
:102860000023036043608360C3600361436183614D
:102870007047002343608360C3600360036143616A
:102880008361C361036243628362C3627047000075
:102890000E4903680A6810B544691C4383691C43E8
:1028A00022F07F43426823F03003234343EA02636C
:1028B0000B60C36882684C681A43054B234013437E
:1028C000026943EA02434B6010BD00BF001000A044
:1028D000FEF7E0FF90E80C000E491A4383681A43A4
:1028E000C3681A4303691A4383691A43C3691A43C5
:1028F000036A1A43436A1A43836A1A43C36A10B5C8
:102900001A434C69044B23401343426943EA824310
:102910004B6110BD001000A000008090044B1A68AD
:1029200010B142F0010201E022F001021A6070478A
:10293000001000A0024B9A68920600D4986170477C
:10294000001000A0024B9A68920600D418617047EC
:10295000001000A0014B1878704700BF201000A0A5
:10296000034B9B68184214BF01200020704700BF32
:10297000001000A0014BD860704700BF001000A0FD
:102980000F4B00211A6842F001021A6099601A6820
:1029900022F0A85222F410221A600A4A5A600A4A07
:1029A000C3F8842002F18062C3F888201A6822F4F8
:1029B00080221A60D960C3F88C10C3F89010704759
:1029C0000038024010300024003000201E4A936876
:1029D00003F00C03042B10B503D0082B03D01B4BC2
:1029E00019E01B4B17E05168536811F4800F5168D0
:1029F00003F03F0318BF164AC1F3881108BF134AFA
:102A0000B2FBF3F3104A4B435268C2F30142013266
:102A10005200B3FBF2F30C4A036093680D49C3F311
:102A20000313CC5C0368E34043609468C4F38224DE
:102A30000C5D23FA04F484609268C2F342328A5C2B
:102A4000D340C36010BD00BF003802400024F40032
:102A500040787D0101000020044B1A6B09B110433E
:102A600001E022EA00001863704700BF003802400E
:102A7000044B5A6B09B1104301E022EA000058638D
:102A8000704700BF00380240044B9A6B09B11043F5
:102A900001E022EA00009863704700BF003802405E
:102AA000044B1A6C09B1104301E022EA00001864DB
:102AB000704700BF00380240044B5A6C09B1104304
:102AC00001E022EA00005864704700BF003802406D
:102AD000044B1A6909B1104301E022EA00001861B1
:102AE000704700BF00380240044B5A6909B11043D7
:102AF00001E022EA00005861704700BF0038024040
:102B0000044B9A6909B1104301E022EA0000986180
:102B1000704700BF00380240044B1A6A09B11043E5
:102B200001E022EA00001862704700BF003802404E
:102B3000044B5A6A09B1104301E022EA00005862CE
:102B4000704700BF003802404209084B012A01D1FA
:102B50001B6804E0022A01D11B6F00E05B6F00F0EC
:102B60001F0023FA00F000F0010070470038024017
:102B7000024A536F43F08073536770470038024036
:102B800082B000230193054B0193019B03EB80006E
:102B90000190019B196002B0704700BF50280040AF
:102BA00082B000230193054B0193019B03EB80004E
:102BB0000190019B186802B0704700BF5028004088
:102BC000431E0A4410B5914204D011F8014B03F89A
:102BD000014FF8E710BD02440346934202D003F8C8
:102BE000011BFAE77047000014000020282C0008A1
:102BF00000140240004000000E00040000140240D7
:102C0000008000000F000400000000000000000031
:102C10000000000000000000C4650008202C00082F
:102C2000E82B000850000000006000400000000198
:102C3000801A0600005F60003C2C00080054014030
:102C400000002000000002402000000005000800F5
:102C50000000024080000000070008000000024061
:102C6000100000000000000000000240080000000A
:102C700001000000000402400400000000040240C3
:102C800001000000000000000018024008000000E1
:102C900000000000001802401000000001000000C9
:102CA000001802402000000001000000001802404F
:102CB0004000000001000000000C02400001000084
:102CC00008000700000C0240000200000900070095
:102CD00001424F4F544C4F41444552000000000008
:102CE000002A2A0000000000000000000047FF004A
:102CF0004C6174746963650069434563756265324C
:102D000020323031362E30322E32373831300050CA
:102D10006172743A206943453430554C314B2D4330
:102D20004D33364100446174653A204A756C203257
:102D30003520323031362030393A35363A3339475A
:102D400002FF7EAA997E5100010592002062016F68
:102D500082470272007011000101470B1047028088
:102D6000470502470580034708014702084711202D
:102D7000470C02470B0247174047050147054047EC
:102D80000C040090470F10470640470501470540D7
:102D900047050147048000044710804705020020D2
:102DA000000800804702014709084717014704341B
:102DB000000C470403470D30475970470E801047F9
:102DC000040200404704080147020702004047048C
:102DD000080147052004474103470B03470D1C47E3
:102DE0001080470901008047020347090847032470
:102DF000472B7847124007470A40470C0400084712
:102E00000E404705014706044704014706044706EC
:102E1000104711800747061C470380470C08470AE4
:102E20000C3020470F30E8470C63C1470C0C30478B
:102E30000F400105470C03C0470C0C3020470D180C
:102E40004702E04704020CB100180038470640472B
:102E5000080C30471001074702010001CD724703FB
:102E600098470F0C3020470D3000F9A0470810009C
:102E700001C04705038047070C30470E300071053D
:102E80004708300001470F0C3020470F580847040F
:102E900001DCA00080470363C1470203C020AF529A
:102EA00047050C3047100803470402E0F5470503C7
:102EB000C0470202E0050FA01047040C3020471263
:102EC00040002020470AC001E007A547060C304714
:102ED000110D470314470B404703054703144702EE
:102EE0000C3020470F900004470220470E17CFA256
:102EF00047020847020C30471030092447022C478C
:102F00000D02CD0FF047050C3020470F108004470D
:102F100003684703010547100C304710110730477D
:102F2000190C3020470D300010470A0147100C30B3
:102F3000470E304702052047023447050247100C70
:102F400030204707044706404704203404ED800042
:102F50000247091C000847050C30470F404705048D
:102F600022FC4702014707A00002C047060C3020A0
:102F7000470903EAF52000404706035CA50018470F
:102F800008401C8F0847050C30470A03D050470201
:102F900040470601F0554703104706200200F0475E
:102FA000050C30204709284703110001E0470320A2
:102FB00038FC8002470A1E8F0847050C3047080876
:102FC000004047033029470402BC03D0470AC047EA
:102FD00003F047050C3020470A1C0F10470829DC76
:102FE000A5003047090E8F0847050C30470C0F47E6
:102FF00009415055002047090200F047050C3020D8
:10300000470D0447065C76EC800247070847020636
:103010008047060C30470802470504470301470371
:103020003CF0470A01400C00F047050C30204708EF
:1030300020470B1C21FAE732004047100C304709AB
:103040000C470B2464F0F7084709028047070C304F
:103050002047141C31CCE720804703383D44470209
:10306000028047070C30470F404705027668FB4750
:10307000024000C0403D4703028047070C30204714
:10308000080C47050147053C63DE800010470C042F
:1030900047040C30470A2047040247052402E8474A
:1030A0000210470601014047020147050C3020008D
:1030B000A100123C20000447021EF06047072000D8
:1030C0001EF04047030D72BD400003428EEF4706DD
:1030D0000C30470503C0C04704F047024000974743
:1030E00003042000F0470401403C470201429C4792
:1030F000070C302047033A3C200647030CF06018C9
:1031000002108000060140024AA5001880000778DE
:1031100015006047020CC96047050C30470503C025
:10312000104704F0470205090747038001D05547BF
:10313000039000401620000142C1096047050C3091
:10314000204703323C202C47031CF04030470280CC
:103150000004470220470501883941470202002543
:10316000ACC02047040C30470503C0044704F001FD
:1031700030080109000C4702404705F00F42820168
:103180000020402547070C30204703323C204702EF
:1031900080001EF040470280E847037C470705781F
:1031A0001547044488002047040C3047040803C82E
:1031B0000001470210F0470371094703964708C012
:1031C0001640000342150020470202001C0C30206C
:1031D0000001017A3C2047040EF0600008704703AC
:1031E000A00601DAA047090A007E8800300002C06C
:1031F000000C3047038D0003C04000243000F0472E
:103200000308FB470240000340F5470901428700DD
:103210002047040C0C30202000013A3C20201004F0
:1032200047070804001000045AA102004000A0470C
:1032300005603EEFA547050C300010070D0803C0E0
:1032400047020247070520470334E001470B1C05EE
:10325000A047020247020C3020040500723C200007
:103260001047060450800447022021EEE20200408D
:103270001810470403601FAAF5470202C0000C3073
:10328000000405470203C0001004470542D8BD2CC6
:1032900000103C767042470240008047030102C0A4
:1032A0002C00F047050C3020000800723C2000A0E4
:1032B00020784703300010470501DCA302304702A5
:1032C000804703C001C047080C3000040B470203CD
:1032D000C00052144704300008033C470234383021
:1032E000A30020400147048101C2C0470C0A723C80
:1032F000204702A03BF9014001404705202C0CF07B
:10330000404703078402470306DEF5E0470A10083A
:1033100003C10001547D69A70040404704020460D6
:1033200000F047028050003C470402BCF1D0104737
:103330000601804702723C20060024017F74400190
:103340004047030647034EA50018470215A3C28055
:103350006002002C91A0470B0803C047023C2E7866
:10336000A01002404707D055470490003C47020197
:10337000401DF3F047070347031215400400366869
:103380007B64403047040CA047020DD10001470286
:103390000723C24702034614ABC420470A0815405E
:1033A00004023C004A58007047040C470203DFE265
:1033B0004705803C47020266C20BC208470A03BCAD
:1033C0001047023C294B7440002847042000281E67
:1033D000F04000021801A3C20004016060AB470C7A
:1033E000043C4703164268A0004047074010F047DE
:1033F00002050800803C47021403B4C70010470AC6
:1034000003BC100C4702035D7A014706A00E60FE64
:10341000A047023001A7A3C2000803469E81A02056
:10342000470A043C0004470202C85A0847071E0323
:10343000C0F54705803C470201601D03F0470C2999
:103440005047021E01D95B10404705800423CCA1E0
:103450000247031123C247041D95E0470B901680D5
:1034600047021C314CA547080202C00247048000F5
:103470003C47043EE1D0470A1B47051F470601C0F1
:1034800047030620E8A3024703B325ED00040166C5
:1034900040ABC42047090A470502470601470526F5
:1034A00070034704AFB694010A0242B507C004474F
:1034B0001064F850104708701AA302B10001D047F9
:1034C00003C00003DDB5E0471164005047083443F2
:1034D000D05300228051A0470380D6C76EE1D04769
:1034E00009081E5BC8104703040AF0404709FE00A4
:1034F000404702198F304002000166A5E0470A0BE1
:1035000000121E806000142800F0470240000747A8
:103510000403F0A04080020007B0470301C24E94AC
:1035200047080180470506470308F0401847021086
:1035300000062000020C0A001947020B3A81816044
:1035400002E68405A020470801470810F04704B7A9
:10355000470240043CC00500028010874001010082
:1035600002601402400447060300080036C9580CE4
:103570000034001AF04030470218000CA14000FE51
:10358000504A0247020120288047030480D0A04708
:10359000060100030A7A05424702144702F0003090
:1035A0004702FB0004408003F0804047044028802D
:1035B0000003400100D080470603000500DE11D85B
:1035C0004702366C1AF060470308000D8000020CB9
:1035D0000A403008000B3801010002000D85E02090
:1035E000470601000F0052E0404702142800F04750
:1035F00003B0070009024702C00548200400074144
:1036000041044702401602E0470A08F680D2100E35
:1036100047021AF0404703184703200400A5400062
:1036200080501175D04703C067A0140447080B09E8
:103630001B28C020470310F04704C900400E3C3847
:10364000C05A480100D887B5F8470303AEE80080A8
:10365000470808019F141447041AF04047028018D5
:103660000400201E2200A54130005C037B080847AF
:1036700002E021CA470A050C56788240470310F041
:103680004703F0E53C470340C05A40104702A7C338
:103690000C04000262DC05470A0D81D6C9504705BB
:1036A000A540470298984702A004301C05408000BE
:1036B00018E04705600685014709050A32054A47B3
:1036C00004405A470399933400400201C00A40471E
:1036D0000210B047030847020105470A0581FE5161
:1036E000D047040AF0403000901000040004027E2D
:1036F0005F40100050E1B8280400E0400FF8124786
:103700000A0B53E04A4705F000300070FD3C04000E
:103710000220E00F48100079098168040002600C63
:10372000C4471114004EA0400240470607C850C0CD
:103730004703904705407EC70008470F020010A0CE
:1037400040804047063BC00542470210D047052352
:103750005DAF01470E06470744470306470203C80B
:1037600050C0180018033E01006000063DC047111C
:103770000447054247050402C005404702188FBCB4
:10378000012047030E824716100001C000044702C3
:10379000674850C0100001E13010470360471830FF
:1037A0000001470204470223E005401047020DE0F4
:1037B00047160C47070547030C0006674850C0F042
:1037C000001017B2012847020780471008470B086E
:1037D000470222E00540204702E7C001472340039B
:1037E000E850C14703F0470402662F90471B10477B
:1037F0000203C005404703D0470401442FB04047AF
:103800001D736850C010470219F56C47020366EE3D
:10381000D0471E42C00540304702ADE11C470201BF
:1038200042AEF080470240470E0447090226036873
:1038300050C00007101DFB08084702068DE8002055
:10384000471038470A0403E0054040003085830CE8
:10385000470508470F04470B040020736850C11048
:103860004702804703C00060208E5420470D044764
:103870000B04000442E00540100051E04703804182
:1038800042650DA0470372009011010101470B1022
:103890004706404705014705400002470608471113
:1038A00020470680470502471208472201000247C9
:1038B00004044711104706404705014705404703E8
:1038C00016000147060447220200200008470208AC
:1038D00047031047243C000C4706304768801047D8
:1038E000040200404704080147030200404704085F
:1038F000014704302004474D0147060447210300D7
:103900008047050247030C471F1E472D024703400F
:1039100047050147174047050147060447030301D0
:10392000470604470610471D8047050247110C3023
:10393000472C0C3020472B0C30472C0C3020472BC9
:103940000C30470E01470C1047100C3020470D0279
:10395000471D0C30472C0C3020472B0C30472C0CCB
:103960003020472B0C30472C0C3020472B0C304795
:103970002C0C3020472B0C30472C0C3020472B0CC4
:1039800030471308000400205547088000424708CC
:103990000C302047120C00200168554047074002B8
:1039A000004047070C3047150400200F470B020565
:1039B000500447040C30204714260168F0C0470922
:1039C000661E855447050C3047180F470DF0804799
:1039D000040C302047150168F0C0470A168F0C47C9
:1039E000050C3047150C47020F470DF08047040CBB
:1039F0003020471501E8F0C0470A1E8F0C47050C20
:103A00003047150C20200F470B0200F047050C3003
:103A1000204714266548F0C04709601C8F0C4705F5
:103A20000C30471620200F470A460200F047050CCD
:103A3000302047156548F0C047080207548F0C0036
:103A40000147030C3047180F470DF047050C302095
:103A5000471206470201C8F0C047076047021C8FA3
:103A60000C47050C3047170C0F470503C0124702DF
:103A70000401B0F047050C3020471501DAF0C047CB
:103A80000423C0470307148F0C47050C304718F078
:103A90004703D9B0A4470280470A0C3020471406D8
:103AA0000008F0470350A780020040470A0C304747
:103AB0001620300F4703D900A047040247080C30F6
:103AC00020471505780F80470250A7800247034022
:103AD0004047070C30471524201B0F470528470D8A
:103AE0000C3020471501F80F804703078002470C70
:103AF0000C3047170D0F4704B020470D0C302047FE
:103B0000140661790F804703078402470C0C304785
:103B10001504200D0F47035000A8470D0C30204717
:103B2000142004F80F804703070002470C0C3047AD
:103B30001506203C0F47035000B4470440050A080F
:103B40008047040C302047143501C90F804703011A
:103B500000024702026000E50447050C30471536B5
:103B60006C1C0F47035000284707588047040C304F
:103B70002047141428E80F80470307040200604719
:103B80000214E05447050C3047166D4CA54703500E
:103B900000204704C0040A088047040C3020471561
:103BA00029415A8047038700024702024702A504C1
:103BB000471B10044000F0470301A9A00004800047
:103BC00042471F207808F047020800BFA02140406C
:103BD000020040471D10042060A54702404702A094
:103BE0004702010040020550471C2007605A8047E9
:103BF00003078002470202601E8556471D0340A549
:103C000047035190B04702014704F0471D01605A35
:103C1000804702D9A3840247020800168F0E470E80
:103C200001470D1C004FA54704A0703C4706F04714
:103C30000E01470D2601E15A80470219B5F43E47AF
:103C4000041E8F0E471C1C20390F47031900B44770
:103C500004028200F1471C2605580F804702F9E351
:103C60008002470360148F0C471C1C3C2F0F470336
:103C7000100034470320020200F1471C2061DB0FD3
:103C800080470280030002470306548F0C471C3C08
:103C9000381C0F4702180090F03C4703028000F1E7
:103CA000471D04C80F8018003DA5E03E0060470294
:103CB0001C8F0C471C3C380C0F47031000283C4756
:103CC000040190F1471D25CA0F8047029005643E0C
:103CD00047041DBF0C470E04470222CF4A60470528
:103CE0000400042047031000188F62E100410042E5
:103CF0001C05A0470E04000467FB40404705040074
:103D0000360447031000981D6CF1024002002C4756
:103D1000021001470604470208284702100025F058
:103D20003C6000424704100232DAC3400040018583
:103D300041410005000381005004470A16A80447CA
:103D40000206067A7C424047060402DFD34800049C
:103D500059F0728147041EE0504710023FE8F247D5
:103D600007801C7AE0A5470220080F3001400001BF
:103D7000C25C05A00401470D100E62DFFA47071070
:103D80002026FC500100C018E13A01000147026EF4
:103D90004713214FF54707014221D90740007D0015
:103DA0000F2811000101C026020414471006EBF68B
:103DB0004707011C05FD036100021987F69D0002FB
:103DC00047021F800420470809470408000628E02E
:103DD000182040470408470202DFE3402000D80BC8
:103DE000656100940142B501470A0847040C002EA2
:103DF00007FA040247050C00042BCCC36070009145
:103E000087BA8900CA020021C20020470F3C001077
:103E1000A0470208470601F0D3410147029FF9512C
:103E200000040002B680404711014EA0470902E895
:103E3000C342020070153EC1470306D5A0A047103B
:103E40000642D0B9404707042830A047031805733D
:103E50002147036037A1470F06000E3BDCB16247E4
:103E600005064703DAA00018007C0FBB09006001BB
:103E7000E035D047020A470810470602CFE0470D59
:103E80000400190F21194702014247040447080E94
:103E900047040E47021BD0470930470304059981A8
:103EA000720D470202470B03000980920447047F0A
:103EB00060C2470604014203400500100801804724
:103EC00003400340470A03000F80174705386CC3BF
:103ED00002470504009E000E0A20100058F0470318
:103EE0004047101814470403F00347081E3C30A055
:103EF00008470290E77F21470306EED4A447090153
:103F000000DE8047030402DA430247073E056EA045
:103F10004703B819FF4147024002B689144709090F
:103F200008941047034040F0024707802C3F5ECBC7
:103F3000470308A9836101470202020F470A0801EB
:103F4000F7470280470260C80A0247060E20060CA7
:103F5000C7104702781BEB0108084702468F084745
:103F6000094B00164047020146387B020100024718
:103F7000053C3C100A47033009807447020363C0C4
:103F80000F470A200012204703BC7AF947030D4768
:103F9000052005DA0A200247020772B4080009402A
:103FA0005E8F081047080B0D941A4247033C00A08F
:103FB00008470508001C294B08002020D005414770
:103FC00002800002C20F470A080B06A5904703694A
:103FD000CAA02047050C0020020C042032801809DA
:103FE000200008C047025C8F084709200E10000817
:103FF000470324300401470504470220CCA1414770
:104000000218B0C0284704020F470C179000800028
:104010001429EA040247050447020378D1408000CE
:10402000D005782847041C8F0847090700D04703AC
:10403000401472D947030147050401CA5B470311C5
:104040000567B840470242800F47080180000A76A2
:104050000080808000767B802000024703060E14DB
:10406000000DA708180159C573BC006047024C8FAA
:10407000084709050EDF00804703237B470A26CE49
:10408000FF094000D9E3384147072047080518DAFF
:1040900047053CE980200038470603DBF747033833
:1040A000A1380147040C00080040470235005013B6
:1040B00047030403C04702266D70400840470404CC
:1040C00000047C7005470308ABA39C204702030152
:1040D0000F040040014020E0A00147030683D047C1
:1040E000022428DA5012470504002423EC470280FA
:1040F0000071B17EBD40404702418F044703467EB8
:104100000D344702014706046410A0470702003639
:10411000DAF0484702500743000147040F04470202
:1041200001639CEC342000098047052065DEA04730
:104130000901FFF4404000D9A720000A4702070008
:10414000CF04470202403401A0470802266650010E
:1041500047094370A04703500FA400204702040101
:104160000F0447042FE00220470826760E0222475C
:10417000070621EC4704980FF420470303808F06BD
:1041800047020140010A4706154001800C62CC47F6
:1041900005C047043D40E740C10050A70300204749
:1041A0000202410F044702020284AA47055A155031
:1041B00001002026FE0847041000804702077CD338
:1041C0004A020081D772000C0801E001CF04008090
:1041D0000042470501800803C047020C41DD20472B
:1041E0000608002E39D00A47030800C028204702DD
:1041F00020010F0400C002004047040D98523C30DB
:104200000240002ACF47070C0006036C4704300722
:104210003028010001C000EF044703029E47050853
:104220000803C047021401E024001047061C207058
:1042300000414703A0C14702404702010F04470461
:1042400037AA0104470219523C30470302DA100230
:104250003002470604EE8063470315310028C0474B
:104260000201EF0447034035040010470403C04730
:104270000303F0470340470506034A1047030803BA
:10428000240020470202400F0400604703880121F8
:10429000804702723C30470368EE402200404703EB
:1042A000060006021E2000180031EF320021604790
:1042B0000201AF0410470223CDE0470603C14704C3
:1042C000EF47034047051401E04705A5FBE047031E
:1042D00006010F0447036004C0804704723C304766
:1042E00003027D804702404706036A0A4703019B99
:1042F0002FF483470203808F048047060100010EDC
:104300000803C0044702404BF1493000080F28045D
:104310004710140500044706030008187A3C3004CF
:1043200047023BCDF040700010470204470610479B
:104330000280470503A18A4704028047060803C498
:1043400047050A40800070FD24470280470D028027
:1043500047050280470401805A3C3040000600FABD
:104360000A40470380470201470D0142C04704014C
:10437000404704038F470203C010470238ED0BC1CA
:104380000002008D28470A010141840001C02782F4
:104390004704068047065A3C30400006027A054929
:1043A0000005470204000E47092A81A047031F9316
:1043B00080470950470203C010002401505F404766
:1043C00002700300404702304703044706400002E2
:1043D000800F0008470820007A3C30000E00637A06
:1043E000A5404702804705044705184704C0006000
:1043F000008F00044709180803C05800042C70E31C
:10440000404702909D0008470E01C00300F0470995
:10441000018B523C300C002C03FCC34200380008D6
:10442000000C470E020014E0F847043FC0470408A0
:104430000803C050470201700500300031F1000C44
:10444000000440470B40022ECA5047041DD080474D
:104450000319523C3020470202DA470230008090B4
:1044600000040020704705784706065415A8470841
:1044700003470303C04702042C6A8140000200077F
:1044800047030447052800F3C2BF800003D280C061
:10449000F0470701804702723C3006010C026F5062
:1044A000401801470306470618180007E29547031E
:1044B000400EE0F8470950000AC0470401DA3C47C3
:1044C000024010CB470402C005444280084706045E
:1044D00002470222470820007840204703016D343C
:1044E0004704184704014850400100704706071C64
:1044F00000084703720070110201014708024706D5
:1045000008470402470A04470220470680470C0177
:10451000470604470401470802C047031047170233
:10452000470608470B084716024706084704024794
:104530000608470620470680471F03000700044778
:104540000B7C471D03470F6C470CA8470502472704
:104550002047080447220240C047040801470302DD
:104560000040470408014705200447058010474CD8
:1045700003470D70471F014703044709D047034015
:10458000473A02471208470D80470A800002470356
:1045900002470580470502470608470620472204D0
:1045A000470D401030C04718067B38470240626D07
:1045B0006140470383DC05470430C0471803DBD064
:1045C000470301AB2022C0470203C000804702100E
:1045D00030C047160103F8EC00B0018047020162C9
:1045E00000060083D6000A00180030C0471703F801
:1045F0003001F0470903C20D1047021030C04716C2
:104600000108805A00B01400AA49A1604003008349
:10461000C447030C0030C0471702002D018008007A
:10462000064B6C0280030003C247041030C0470AE7
:1046300080470D14EC50104702A2EDF5404703836C
:10464000CC054702800030C047193AD8F04703A193
:10465000E420470303C2008B01001030C04716015D
:104660000A805F804708030083C60847032030C0E4
:104670004717210028104708020003C00547031010
:1046800030C0471002470980470502470483C647E8
:10469000025C470230C0471A10470503C0470303B6
:1046A000C2470280001030C0471708096947074019
:1046B000470383D60581470330C04718215D47076C
:1046C00020470303C0000A47021030C04717088084
:1046D0005F18104707100083DC4703800030C04795
:1046E0000901470E227A00804707600003C2470293
:1046F00001001030C0471704000A1847024010F1AB
:10470000296047060A470330C04718015047030491
:104710000F00014047091030C04717043C585010A3
:10472000018010F16A06804704014702180030C07A
:1047300047183C10508047020F0041404709103095
:10474000C04717043C5878A0470210F121404703A6
:10475000A906F38000480030C047183C10584703B2
:104760000F004002800020193FE547028C1030C046
:104770004717043C5C470410F121604047028BACB2
:10478000E00A470330C047183C1000C047020F0042
:10479000400280002002A7B50A47021030C0471728
:1047A000043C5C470410F160470490B7884704302C
:1047B000C047183C1047040F47050222EFF5470297
:1047C000201030C0471708024B9980470210F16053
:1047D00047048BAEF81B470330C0470901470D0261
:1047E00010DA1047030F004047030202A5A50A474D
:1047F000021030C0471708025A470410F1684703F7
:1048000020A907D19A020C0030C047170122EB47BC
:104810000220000F47048000193EA58002081030D6
:10482000C0471708826B470410F1284704A93CE0F1
:104830000A470330C04718115D47040F0040470284
:1048400080022A26800002001030C04717183DC0A1
:104850004704169947058001B50A08470230C0474A
:1048600012028C000800083C20470303096B47052F
:104870003FC1ED9047021030C04709056047081C52
:104880004702604705018010F1624702060083DE9F
:104890004703180030C047094047080280304706E8
:1048A0008000010F0041C0470303C047041030C01F
:1048B00047130C7C00304703100080800AA1384762
:1048C000020300A9408047020C0030C0471202C218
:1048D0007800304703084702C00AA0404704294037
:1048E0004703081030DE4710084702404709C06000
:1048F000F180470483C4470530C2470F0114000309
:10490000470A4000F0800008470203C20D0B47022F
:104910001030CE47090847095C470A2A500447036C
:104920000183C4470240470230C2470908470620B6
:1049300002024702804706200045A034470280005B
:1049400003C20947031030C00700A0470F804E780C
:10495000470720002A50470902470230C04709088C
:104960004708B24278470905A03C40284708103064
:10497000C04712800E470C024702808083D647054D
:1049800030C047090847062000F24000084704D01D
:1049900000204703024000800003C04702020010CD
:1049A00030C0074703020F78044702204708540528
:1049B0000030470680470A1C000C0030C047040244
:1049C0000F080247082000B3823A8020470680473C
:1049D0000580470410A20447071041F70028001083
:1049E000470380A0470508000803790004470959D8
:1049F00081A50A40470ADFB4404705714706080011
:104A0000608369D0B04709198D0D9047090224834E
:104A100080280044090AF900A00180470308000823
:104A20003DC080E0018020F5470306005A64A0479E
:104A30000A02E7B3C0400010222FDA11B047050880
:104A400047023C2071B04702A0F080038047021A61
:104A500074470B02AA77144703014148504702806C
:104A60004704304704A010002A57A86047035A445F
:104A7000850A470902AA0C022C4702014000D8B05F
:104A800000804704204703F147030F50F5C0470358
:104A90001A640090470A1892D428000101406A5015
:104AA000104707083DC030470320F5806047035A90
:104AB0004488470B341EB46C470223401BD8F04790
:104AC0000608203C0030470320F08047041A6501A7
:104AD0000B470940053EC04704046B8047020800AD
:104AE00020470814470302000347020CC5A8000D25
:104AF000404707080807C047040358104702020050
:104B00003C4708084704404703332CBB0E0080474E
:104B1000080112862800014294DB4703C0470F08B2
:104B2000470780470A1E8040470202003B00900072
:104B300080471028470660470850A55EE0600002E5
:104B400008BBDA80E0470701E94E5180470610476D
:104B5000023C1C07470B85068447042A6EF0470673
:104B6000744702AA78F847072847023C02078047A3
:104B700009025A005470007047038047070108F487
:104B80006A470420F18247020240029DE747028003
:104B9000470702A503424000304703F000024707E1
:104BA000980B470420F001C0470280028300800177
:104BB0004708030F52A047030C3E6A47090294DEE0
:104BC00018470A5414850A470AF0983C470303C360
:104BD00060470901541FD0470990144702904709C4
:104BE000030F13804702600C3C4E300001804706E3
:104BF00014C8470201804703E00846005A45E047D1
:104C000002184708F0470503C0470A02BC1CD047FA
:104C100006220020001A7400084709030F13A60497
:104C200047020C3C4A9810470505000294DD51E00C
:104C300000100AF184470443C48047020C4708F07F
:104C4000043C20470203C0101080470502000154B5
:104C50000909470305F0A047043C010D0B000C4770
:104C600007030F12806030000C3C4AB180C8470730
:104C700015CA5004470220F580038003005A65E0FE
:104C800047020C4708F004470403C0101000144703
:104C90000602BC1C084704F0470302001A54000B2C
:104CA00000044707030F178047030C3C5E47028050
:104CB00047060294CDF9F0470903C4470CF04705B5
:104CC00003C0470A01541F70D0470603470203C0C0
:104CD0004708204702030F168047030C3C5A000187
:104CE000C8470714FAB8E047080183DE47021C47AB
:104CF00009F0470503C0470314470602BC3CB890BF
:104D0000470983C0470B02AA17A06047020C3C5A10
:104D1000018047060101E8FF71C04705078047048D
:104D2000010010804708AA0404470303C010470A83
:104D3000542C08470604470680470C200400200A2C
:104D4000A85E181400C047040108F54C704704A77A
:104D50006000044705080008470A0420001002A864
:104D600010008A0040470404006419F8F0000100B4
:104D7000A0470A08470E083D6000044705200008C8
:104D80003DC047048005E000380004C3FCA0471183
:104D9000483C00F04708083C47062BA342D00004DB
:104DA0003C3E470B020F78470360083D601000014E
:104DB00080470A05804019B006000600C3C4E047DA
:104DC00002184707020F084704083C00F8470B7019
:104DD0000008470201EB404702243C471230083CE0
:104DE000E070470280470440083DE03047028028D9
:104DF00045E04704C3C4A981470F22083C200800AE
:104E000014C04705083C204703C0242BA002C0471C
:104E1000023C0101084709020F304704083CE00149
:104E2000F04707083C604703204009B047023000C4
:104E3000C3C4A9984709020F4705083C2001E04771
:104E400007083C20470521EB4047033C0101470D83
:104E500020044702183C6000800847040547090504
:104E6000E2E0284702C3C5E0470D3C384702083C52
:104E700020014705024705B04703808BA060470328
:104E80003C4713083C40F84708083CC047042A0147
:104E9000A440470201C3C5A04711083C20F04708C1
:104EA000083C20B047032050A04703043C471202AF
:104EB000083CC047070100083DE0470501B14047F5
:104EC00003C3C5A0184710083C470A083C4702C066
:104ED00047033B7C2047033C0103470D0E010020A4
:104EE000083C604703804705083CE0470384000115
:104EF0002447020200AA85A101000C470B02800092
:104F0000083C2000044707083C2010E1470202004B
:104F1000B447042A8100080004470272009011037C
:104F200001014708024706084704024708078004B2
:104F3000470220470680470C014706044704014703
:104F40000D10472A0847160247060847040247067D
:104F500008470620470680471F02470304472903E6
:104F60004729A0472D10471E02004047040801476B
:104F70000302004047040801078047032004470557
:104F80008010474501470603470D20471802470692
:104F9000034703044709C0470340472B384721080C
:104FA000470B400080470A804705024705804705B8
:104FB00002470518084706202C471101470F0447F0
:104FC0000D400030C0472B1030C0472C30C0472B5D
:104FD0001030C0472C30C047100447180100103073
:104FE000C0470F80471C30C0472B1030C0472C30C3
:104FF000C0472B1030C0470E10471D30C0470A0273
:1050000000140B471D1030C0470C28E1471E30C06C
:10501000471B04470F1030C0471B0A471030C047DA
:105020000B20280B471D1030C0470C14E1471E30E1
:10503000C0472B1030C0472C30C04725330690475F
:10504000031030C047242031A480470430C0472BD0
:105050001030C0472C30C047253C0247041030C0F8
:10506000472304803C14470530C04708804721800F
:105070001030C0472901400030C0472701470310C6
:1050800030C0472C30C0470A80471D0A4702103005
:10509000C0472801470330C0471D0300F0470705FC
:1050A00047031030C0471FF147070D9A470330C030
:1050B000471702A809704705404706010800041079
:1050C00030C0471180470501544147041000796002
:1050D0004705080100080030C047150447023C4757
:1050E000060B404703802A81000847021030C04762
:1050F00015020007C05847041008684704AA85E154
:1051000099470330C047183C1047050301428047C8
:10511000023C47051030C0471707C04A4704100833
:105120006A06C04702C3C5A0470430C0470F044702
:10513000053000025A40470503014047033C47053C
:105140001030C0470F0A4707065848470410086B3D
:1051500066804702C3C5E00080470230C0470FF0B9
:1051600047083C100847040B41428047023C014776
:10517000041030C0470F10470707C05A38470310C4
:10518000002A06C04702C3C4E018470330C04711D5
:10519000C04705025A500147040B41428047023C78
:1051A000010147031030C0470E50470280470506F3
:1051B000585E71C0470210002B66C04702C3C4AFDF
:1051C00000A0470230C04717025A50470503470462
:1051D000013C47051030C04710018047050658487C
:1051E00070E04702100028470301C3C4E0470218DB
:1051F0000030C0470B083C470901000140984704B4
:105200000100034047023C3647041030C0470B08FA
:105210003D60470904470238E0470210002800407B
:105220004702C3C4E7470E3C47021010D9470D049C
:10523000470506C04702080247112000034B470DEF
:1052400002470502800010081CE0470D02000847D5
:10525000040200204703028047041047041BB842A1
:10526000C047021080900902470B1C470C01470AF7
:10527000073E47031014979598471301E04707012D
:105280006BCA999047093016B500024713F04707DB
:105290000160699990470506804702103488470FDE
:1052A0000847040100204704040002A8100847032F
:1052B0000A008364471580470401E04705020202A3
:1052C000A85C1847030A037942804718D9F04707BA
:1052D00002003C1000E04704704704069E901B4704
:1052E000110B4B80E0470707C05C00100004080763
:1052F000B0470301A94F800A470E053203D42008A6
:10530000B002470508003C47020A470240A0804718
:10531000042801DD80470F3003D56A7880024704F6
:10532000300007C05C00044703A37847051C95477D
:105330001E3C4702A047090E01AD1A470E01604707
:105340000378470817C05C00104708100617900A3A
:1053500000184707020F4705A0014C4706029001BD
:1053600047021000E04702080B38470534A01B47EE
:1053700009920F784705824D470601470204000C49
:105380000010470303BC000447020216950A4711A8
:1053900003D047022047040604003C204703202096
:1053A000F080470402378009471004001A788147CB
:1053B000050104183C6047032020F7816680020144
:1053C000802CE04703023FC04709024703D070002A
:1053D000204704024706202020F00142808000136D
:1053E0008299090200443FC04709010004001A8164
:1053F00080470B01002020F30366C00012A346057E
:10540000471340470A3C470280003020F047051E02
:10541000810029471004021A01E0470604183C6085
:10542000470420F780E04702101E8CC0470E01475A
:105430000301C009E02847097008002060F080449B
:10544000008000084E810A0080470B0247020402D8
:105450001A79F004470B200020F380070080000435
:10546000B408471202D050A04707603C20470320F1
:1054700060F0804702500010038D471104000A506D
:10548000A0084706183C4047032020F747041000B7
:105490001D80470E01470203C25010A04707229407
:1054A00047048060F080470202003040C79F470DEC
:1054B00002800007C0CAD04707081A9408470201B3
:1054C000E020F74703031030941F0E471003C0601D
:1054D00047020447050C02940050A0006060F047AA
:1054E000052001ED80471007C1EE01E08047050867
:1054F0000A94084702010020F7470306100014A58C
:10550000470218470B01470203C040508447060C6E
:1055100001680C50A0003860F0470502810D1F4063
:10552000470C02470207C0EA00B84705020A0A947E
:105530000100A0470220F74702084000029EE00A4F
:10554000471042A8103080004047112047040B4705
:10555000100AA85A001000C0471150471543C01048
:10556000008047083C470401010F340280470201D4
:1055700042000E47100C3C5A01904707083CE04798
:10558000050731404702208155E0471123C0003014
:1055900047093C00080040008000A0000347160CAB
:1055A0003C5A00014707083C60718047035120477F
:1055B000070E471023C0470201C047073C20008068
:1055C00080000FF0A14047170C3C5E4709083C40A3
:1055D000019047028FA5200280470401471123C094
:1055E000101047093C204703010103B80010004098
:1055F0002042E09047100C3C4A99804707083C4005
:105600004704020747022000100056879E471023D8
:10561000C0101047093C00084702C047020140473C
:10562000031C16B147110C3C4A984708083CC05867
:105630004702804707102DD0471143C0470B3C4716
:105640000280004047040347160C3C4E470201808D
:105650004705083CC0001001470520470718470EC2
:1056600043C2E0470A3C2010470501428047050D30
:1056700047100C3FEE4709083CE098470602804778
:10568000050110470C40471A630029400010002014
:10569000470B7047088047111200A9408018470D3A
:1056A00040024704084727200147043847120647AD
:1056B00006180040472503004003C2001047270199
:1056C000470283D60018470E30470401470C0447B1
:1056D0000540471B80470B02470402470240470F23
:1056E0000F06804703083C000147050285470B046D
:1056F0004702040281C047090102007A804703087B
:105700003D40008047040102470B074703A804B14E
:105710008A470D280002083C20014702C0470408C0
:10572000403C00088000802A5034024702840281F5
:10573000E108470C064703083C6001E000C047034E
:105740004000183C605010148025A04702404702DA
:10575000E804B981470F50083C470B3C2001470241
:10576000402AA040470201000280C0471050083D77
:10577000607A0001804705183D4000A001002AA77B
:105780003047020405E804F00A2018470C7000486E
:105790003C470702700023C000700447022E7B388C
:1057A0004703060294E00E4710083CC047090BC1AE
:1057B00040000A470222402800054702E826B001BF
:1057C00047031006B04704807E8047030154184702
:1057D000080800B01908D04705034047022A81474E
:1057E0000580BEF198470202027680384702229572
:1057F000EA01E100804704010A75E971F0470401FC
:10580000E04002012A96E7804705D010470280AFAA
:105810000654300002017C0B470601470202F43CAB
:1058200047048050BC6047020430E6D047048286BB
:10583000B01C4703053376684703147D4707800192
:105840000141791808C00040A187E0470391E7B102
:105850008047032004A14704841282284702096874
:10586000090880470702BC2A7180470401E047030A
:105870003E820919470380A5E847030200F20E6C37
:1058800047020A940139E1C0470714FA01C04705ED
:10589000E047033E94C009470303C14705AF0E42EA
:1058A0006002020968087047080154087047034005
:1058B00000FC470515910F470343C4A047030405A7
:1058C0003A462805000A940080470802955E800841
:1058D0000004001164470554A8470403C1010018DF
:1058E0000008550A470420141C470601470202BC61
:1058F0003A7080470205008002470303C0001E473C
:105900000343C5AD9A4703A51F86470302BD6950EF
:10591000A0470580470215EC80B0470205012140F1
:1059200040470283D6000A470303C0050A470340E5
:105930003604204702083C200847028047020247FD
:1059400003D82F08F04702A8503C002047023C0033
:10595000D59B470343C4880147020220D2A0644775
:1059600002083CE0504702C047040148D47A701056
:1059700000042475F847043C15C38A470303C04755
:105980000310000403CC004040083C470804000119
:10599000C019D847030500BC0020008028B5918AB3
:1059A000470343C5A01E001042205220600050282B
:1059B0003CE07980018047040102E8EBB8000180F7
:1059C0000007A1600006001407E947021847023DDE
:1059D000000D000200050AC03C47047C10F0470798
:1059E00002A809D0A540002CBD746247022030CE29
:1059F0008D47044021A01B4703A5575428020020CF
:105A000040F980B0470401470202955D80084702D3
:105A10002C3DF76040200020F4950A470472008076
:105A2000110062002F8247020103470410000800A2
:105A30001010020204002200202000080424044761
:105A400007080447032004002020202400082C0419
:105A50000C0C47030410100C001000084703080842
:105A600047030830003030040022260604080004F2
:105A700004000447042008000C000828000C00085B
:105A8000002808001008082808470228282847028C
:105A90000C10101024000224242C2C0400282C218B
:105AA00001080011301020000422022247032020A8
:105AB000203004083010001008000404040400041E
:105AC00000044706080004080808470208470224A3
:105AD000240400042C2C282847022101211004084A
:105AE0003010201047022000202008042020200031
:105AF00004470404080004040404001010101010EB
:105B000000060810080803024702040408020424DF
:105B1000242404002C2C2820020021012100020A48
:105B200020002800080228282030040030301020EF
:105B30000002470204000A020404001400061010C8
:105B4000100804470208080008020C040C2C02028A
:105B50002C2C2C2C0006282A2A470208220022007E
:105B60000C02200220204702202030300202507018
:105B700040000A0E0C080C0447030400100808102B
:105B8000100212040002202020080824242400020D
:105B90000247040A0E4703020447020624060808C7
:105BA0002C2428280202201030100E0A2010280869
:105BB0004702280020200A08203030180400021A6A
:105BC0000A040A0A0C040C0C470208082808020CF4
:105BD000080828080C02280A2802000808022008E1
:105BE000080020282010000C1010041008020404E3
:105BF000280C040828202121080031303020060E0E
:105C0000222222200E0620470220040C1010100031
:105C10000A4702040404000C040447020A02470273
:105C200008000608080A020808000604060402061E
:105C3000082A28470321213130060A30302020026B
:105C40000220202000080400201000060010001090
:105C5000000C0400040404061614101010020618A8
:105C60001008080147020804040A02040404060498
:105C7000082A0C2A220A0223232322000822222A8D
:105C8000200A02282A301004001010000802020026
:105C900008080008000C040C0C0206180818180468
:105CA00000081808080A020C0C0C0600080E042252
:105CB0000E0A06222A22220008222222220C022276
:105CC0002222220200320010100002405040000246
:105CD0000C08080C04080A040447030810101212E8
:105CE0000400024702200E04240424200C0E0200AB
:105CF0000202020C02020202040206020606020866
:105D00000A262A08080B30303030060820202828C0
:105D100047028200800103000228282800020808A8
:105D20002818180E091A1A0A080208080C0C0C0088
:105D3000020C002208000E020A22020603020222BE
:105D40000208080202220208082220301002041071
:105D500014040408000400080804080800012102D3
:105D60000011301020080E022202000A0847050226
:105D7000100010100247021000040A0C0404000670
:105D8000080802000A0206000A0A020E0A000606B5
:105D9000060200040A0A0A02020013011130040A72
:105DA0000030002002470508061047030647050299
:105DB00008100004470314141010000218101818DB
:105DC0000147020804060200060606020C080A0A39
:105DD0000A00080A03010320470202200A020A00FF
:105DE0001A0A1A120400081A08080002080808080B
:105DF0000800080C0C0C02040C0018100400101809
:105E000000100002040606060808060202000A0C3A
:105E10000002000247032000220C020002120002CE
:105E20000012121202470240424047020C080808C2
:105E30000400020404044704101212040012470371
:105E4000020004060602470202020202470202475B
:105E5000020604020406060002000A021A0A0001F1
:105E60001212003204470220082000020808080825
:105E70000200080008100403121A12084704040262
:105E800002020606020200042202020006010002CB
:105E9000000247022200020A47023A2A321A02048A
:105EA0000412040447040808040008000101020069
:105EB00011101047020402020247080247021010A4
:105EC000020010100010000604060602470202023B
:105ED0000A000600080A040200020404000200048A
:105EE000080A0A10020013131302044702024706AD
:105EF0001047020647021000060010001047020A71
:105F00004702144703141410040002180018180064
:105F10000110120616020006060200040008080816
:105F200047020201010147041018100200181A1A52
:105F30000A04000A020802000200080008470404DC
:105F400004020404040010040010101210000216D1
:105F5000060606470302470202040808084706101F
:105F600004021000101002001002020204000202DB
:105F7000000200080808080800020404040447049A
:105F80001202040012101012020006160602470345
:105F90000247060400040004040014020018181844
:105FA0001A0001120202020400024702080002085D
:105FB00008000802470504011202121047021012DD
:105FC0000612000206060006000447022000060131
:105FD00020002047041018104702383A320A020401
:105FE000060606044702110162003F8247020103D0
:105FF00047080247080247060101470620204706D6
:1060000020204706042047064004470740470E85E6
:106010008447070147068047088047060202470673
:1060200002470802471E04470804471E0404471E8F
:106030002047072020470620204706014708014740
:1060400036010147164247084247060202470E2121
:106050002047062021470610204706141447065003
:1060600050470610104706101047069511470610B6
:106070009447069090470610104706021047060204
:106080000247260404472604470804471E20470702
:1060900020204706202047060101472E014708011E
:1060A000471E424247070247063020470630304726
:1060B00006111147061410470650144706105047A2
:1060C0000610104706111047061011470694944712
:1060D0000610904706101047061210470612124786
:1060E000061010470710470E04470804472E040403
:1060F000472E202047062120470701472601014758
:1061000008820080010347205202470630524706AA
:106110003030470610104706111047060415470691
:10612000404047160101470E84470804470E1202FB
:1061300047061210470610124706101047061010A7
:1061400047060414473604470804472E2020470614
:106150000121471E01470801471610470712104743
:1061600006301247067272470710470E0447074170
:1061700005470740470E0147080147160404470634
:1061800002470802470E0202470610470710104751
:1061900006101047061010470710476621204707D2
:1061A0002147160101471610470710104706121223
:1061B00047062030470642204707424716414047DE
:1061C0000701470E0101472602024716024708024F
:1061D000470E104707101047061010470710475E7C
:1061E00020470721214708110262002F8247020140
:1061F0000347081B1B47041F1B4704041F47101BB2
:1062000047051B1B47041F1B47041F1F47101B1B71
:1062100047041B1B47041F1F47041F1F47051B473D
:106220000A1B1B47051B4704040447041F1F47059F
:106230001B470A1B1B4704E4FB4704E4E447041F15
:10624000FF47051B470AF9194704E4F94704E4E44A
:106250004704F7F7470513470AF9F94704E4F947F4
:1062600004E4E44704F7F74705F3470AF9E947046C
:1062700014FD47041E1C4704F7FF4705E1470AE9E0
:10628000E947041CFD47041E1A4704EFFF4705E1D8
:10629000470ADDC947041EDD47043E3A4704BDBF37
:1062A0004705A9470ADDD94704A2FF4704A6A2472C
:1062B00004BDBD4705B9470AFFDD4704A6FF4704F3
:1062C00084864704BDBD470404BD470AFFFD47045B
:1062D00006FF4704040447043D3D4704043D470AC4
:1062E000FFFF470406FF470404044704FDFD47047D
:1062F00004FD470AFBFB4705FB4704244705FDFD5A
:106300004705F9470AFBFB4704FBFB4704FFFB4734
:1063100004FFFF4705FB470AFB224704FBFB47043A
:10632000DFFB4704FFFF470522470A22024704FB21
:10633000FB4704DFDB470426FF4705224780028234
:106340000080010347022C2C47041F3E47041F1FF7
:106350004704CCDE4705C8470A3E2C47041F3F4789
:10636000049F1F4704DEDE4705C8470A3F3E470437
:106370001F3F47049F9F4704DEDE4705DA470A3781
:1063800036470401374704898147045ADA470552E2
:10639000470A76364704C1F64704A9814704FAFA4A
:1063A0004705D2470A74744704C1F44704A9E94772
:1063B00004F2FA4705F2470A74744704E5F4470407
:1063C000EDED4704F2FE4705F2470A7474470427CF
:1063D000744704CF8F470476FE470570470A7474EC
:1063E00047041F7447049F9F470474F6470574478A
:1063F0000A746447041B7447049B9B470476F64762
:106400000574470A60604704197047048999470476
:1064100076F6470576470A606047040960470489B5
:1064200089470476F6470576470A64644704096C91
:1064300047048189470476F6470576470A7676470A
:1064400004097E47048189470476F6470576470AA2
:1064500076764704297E4704C189470476F64705C6
:1064600076470A777647047F7F4704F7FF4704772C
:10647000F7470576470A776047045F7F4704B7FF11
:10648000470477F7470560470A612047045F7F4765
:1064900004B79F470461F747054047800211036234
:1064A000003F824702010347838282008001034745
:1064B00083822244B2010600470000000000000071
:1064C0000000000000040240000400000A0009006F
:1064D00000140240000400000A000900000C024001
:1064E000000800000B000900000802400004000042
:1064F0000A00090000100240040000000200090028
:1065000000000240020000000100090000100240EB
:106510000080000000000000001C0240200000007D
:10652000010000000000000000000000000000006A
:10653000000C024004000000010000000000000800
:106540000080000800000108008001080000020827
:10655000000004080000080800000C0800001008F3
:10656000000014080000180800001C0800000800C3
:1065700010001800200028003000380040004800BB
:1065800050005800000000006410B71DC8206E3B8A
:10659000AC30D9269041DC76F4516B6B5861B24D2A
:1065A0003C7105502083B8ED44930FF0E8A3D6D694
:1065B0008CB361CBB0C2649BD4D2D38678E20AA0FC
:1065C0001CF2BDBD4932435F504D49435F4D4147C9
:1065D00000537475636B20627574746F6E207265FE
:1065E00067697374657220697320696E76616C697E
:1065F000642C20636C656172696E672E004275744D
:10660000746F6E2069642000697320737475636B06
:106610002100427574746F6E2077617320707573FA
:10662000686564206F6E20626F6F742E20427574EF
:10663000746F6E20636F756E7465723A20004469E2
:1066400073706C617920627573792D77616974203C
:1066500074696D656F757420657870697265642101
:10666000004650474120636F6E66696775726174BA
:10667000696F6E206661696C65642E004469737091
:106680006C617920696E697469616C697A656420EE
:106690006166746572200020726574726965732E7C
:1066A00000446973706C617920696E697469616C0A
:1066B000697A6174696F6E206661696C65642E0029
:1066C000435245534554206E6F74206C6F7720649D
:1066D0007572696E672072657365740043444F4E2E
:1066E00045206E6F74206C6F772061667465722030
:1066F000726573657400435245534554206E6F7440
:1067000020686967682061667465722072657365C8
:10671000740043444F4E45206E6F7420686967686B
:106720002061667465722070726F6772616D6D6949
:106730006E6700456E61626C696E67203676362042
:1067400028446973706C617920564444432900459C
:106750006E61626C696E67203476352028446973F7
:10676000706C617920564444502900446973616219
:106770006C696E67203476352028446973706C61CB
:10678000792056444450290044697361626C696EF3
:1067900067203676362028446973706C61792056FC
:1067A00044444329002E2E2F7372632F647269763E
:1067B0006572732F6932632F6932632E63002E2E48
:1067C0002F7372632F647269766572732F693263F7
:1067D0002F6932635F68616C2E63004661737420B9
:1067E0004D6F646520506C7573206E6F74207965F1
:1067F0007420737570706F72746564002E2E2F7321
:1068000072632F647269766572732F706572697036
:10681000685F636F6E6669672E63006164647265AA
:1068200073732000206973206F7574736964652029
:1068300073797374656D20666C6173680066616955
:106840006C656420746F2065726173652073656385
:10685000746F72200050726F6772616D206661699B
:106860006C6564204000496E76616C6964206669DD
:10687000726D7761726520646573637269707469A3
:106880006F6E2100436865636B73756D6D696E672C
:10689000206669726D7761726520757064617465D8
:1068A0000043616C63756C61746564206368656343
:1068B0006B73756D3A2000496E76616C6964206671
:1068C00069726D776172652043524320696E20536F
:1068D000504920666C61736821007072765F657242
:1068E0006173655F6F6C645F6669726D7761726515
:1068F000007072765F77726974655F6E65775F6648
:1069000069726D77617265005765277265206465ED
:10691000616400436865636B73756D6D696E6720B4
:10692000002062797465730D0A00436865636B73B8
:10693000756D202D2077616E746564200020676F6F
:106940007420004F757220696E7465726E616C20E0
:10695000666C61736820636F6E74656E747320611A
:106960007265206261642028636865636B73756D6E
:10697000206661696C656429212054686973206907
:1069800073207265616C6C792062616421004F75BF
:10699000722070726576696F7573206669726D77A3
:1069A00061726520757064617465206661696C65EB
:1069B000642C2061626F7274696E67207570646107
:1069C00074652E004E6577206669726D7761726519
:1069D00020697320617661696C61626C6521004C8D
:1069E0006F6164696E67207265636F766572792086
:1069F0006669726D77617265004661696C656420D5
:106A0000746F206C6F6164207265636F7665727954
:106A1000206669726D776172652C20737472696B80
:106A200065206F6E652E2054727920616761696EF2
:106A30002E004661696C656420746F206C6F616420
:106A4000207265636F76657279206669726D776111
:106A500072652C20737472696B652074776F2E20B9
:106A600054727920616761696E2E004661696C65B8
:106A70006420746F206C6F6164207265636F76654B
:106A80007279206669726D776172652C20737472F9
:106A9000696B652074687265652E205341442057E8
:106AA000415443480048415244204641554C54000B
:106AB00065786974207374616E646279000D0A0DE3
:106AC0000A0D0A00E29688E29688E29688E29688A5
:106AD000E29688E29688E295972020E29688E296F0
:106AE00088E29688E29688E29688E29688E2959710
:106AF00020E29688E29688E29688E29688E2968876
:106B0000E29688E2959720E29688E29688E2968857
:106B1000E29688E29688E29688E29688E29597E285
:106B20009688E29688E29688E29688E29688E296CF
:106B300088E2959720E29688E29688E29688E29627
:106B400088E29688E29688E29688E29688E29597AF
:106B500000E29688E29688E29594E29590E295901C
:106B6000E29688E29688E29597E29688E29688E235
:106B70009594E29590E29590E29590E29688E2965F
:106B800088E29597E29688E29688E29594E295905D
:106B9000E29590E29688E29688E29597E29688E2FE
:106BA0009688E29594E29590E29590E29590E29530
:106BB00090E2959DE29688E29688E29594E295901F
:106BC000E29590E29688E29688E29597E2959AE2BD
:106BD0009590E29590E29688E29688E29594E29507
:106BE00090E29590E2959D00E29688E29688E29682
:106BF00088E29688E29688E29688E29594E2959DEE
:106C0000E29688E29688E29591202020E29688E23A
:106C10009688E29591E29688E29688E29688E296D6
:106C200088E29688E29688E29594E2959DE29688BD
:106C3000E29688E29688E29688E29688E295972026
:106C400020E29688E29688E29688E29688E2968824
:106C5000E29688E29594E2959D202020E29688E2D3
:106C60009688E2959120202000E29688E29688E2BC
:106C70009594E29590E29590E29688E29688E29566
:106C800097E29688E29688E29591202020E2968805
:106C9000E29688E29591E29688E29688E29594E2FF
:106CA0009590E29590E29688E29688E29597E29632
:106CB00088E29688E29594E29590E29590E2959D1F
:106CC0002020E29688E29688E29594E29590E295FB
:106CD00090E29688E29688E29597202020E29688B6
:106CE000E29688E2959120202000E29688E296883C
:106CF000E295912020E29688E29688E29591E295CD
:106D00009AE29688E29688E29688E29688E29688E9
:106D1000E29688E29594E2959DE29688E29688E272
:106D20009688E29688E29688E29688E29594E295C3
:106D30009DE29688E29688E29688E29688E29688B6
:106D4000E29688E29688E29597E29688E29688E253
:106D500095912020E29688E29688E2959120202065
:106D6000E29688E29688E2959120202000E2959AAA
:106D7000E29590E2959D2020E2959AE29590E29529
:106D80009D20E2959AE29590E29590E29590E295A9
:106D900090E29590E2959D20E2959AE29590E29599
:106DA00090E29590E29590E29590E2959D20E29593
:106DB0009AE29590E29590E29590E29590E2959016
:106DC000E29590E2959DE2959AE29590E2959D205C
:106DD00020E2959AE29590E2959D202020E2959AF6
:106DE000E29590E2959D202020004C61737420660E
:106DF00069726D7761726520626F6F74207761735D
:106E000020737461626C653B20636C6561722073F2
:106E10007472696B657300486F6C6420646F776E81
:106E2000205550202B204241434B202B2053454CD2
:106E300045435420666F72203520736563732E209E
:106E4000746F20666F7263652D626F6F742050528D
:106E500046004669726D77617265206973206572BC
:106E600061736564005761746368646F6720636170
:106E700075736564206120726573657400536F6675
:106E80007477617265206661696C757265206361F3
:106E9000757365642061207265736574004661696D
:106EA0006C656420746F20737461727420666972FB
:106EB0006D776172652C20737472696B65207468DC
:106EC0007265652E004661696C656420746F20737D
:106ED00074617274206669726D776172652C2073BB
:106EE0007472696B652074776F2E004661696C65FA
:106EF0006420746F207374617274206669726D7798
:106F00006172652C20737472696B65206F6E652EDB
:106F100000466F7263652D626F6F74696E672072D1
:106F200065636F76657279206D6F64652E2E2E0015
:106F3000456E61626C696E67207761746368646F27
:106F40006700426F6F74696E67206669726D776162
:106F50007265204020002E2E2E0D0A0D0A00426F71
:106F60006F7420626974733A2000536F667477619E
:106F70007265206661696C7572653B207265736528
:106F80007474696E6721004153534552543A20008E
:106F90003A00415353455254004153534552544EC5
:106FA000002A2A2A20575446200053544D333200D9
:106FB00053544D3332207065726970686572616C2C
:106FC000206C696272617279207472697070656494
:106FD00020616E206173736572740069746F612043
:106FE00062756666657220746F6F20736D616C6C7C
:106FF000002E2E2F7372632F7574696C2F736C655E
:047000002E630000FB
:10700400FF00000000010203040102030406070854
:04701400090000006F
:0400000508000200ED
:00000001FF
